:020000040000FA
:060000000219FD02031CC1
:03000B0002008D63
:03001300020535AE
:03001B0002009050
:03002B000202D1FD
:03005B0002054457
:030073000203097C
:100080000406080C10182030406080A0C0054032E3
:10009000C2AFC2A853E6EFC28E856B8BC0D0D2D35D
:1000A000C0E0C0F0C2CAA8CCA9CDD2CAD2AF758A6E
:1000B00000C3E8956CF8E9956DF9C3E913F9E81305
:1000C000F8E5666007C3E913F9E813F8E97025E875
:1000D000956E4020956E501CE582B410177C007B15
:1000E000007A007908900000A86AE5667004C3E809
:1000F00013F801FD900000D2A8D2AA61E7E0FDC389
:100100009CC39840EF98EB33FB0582E0FCC39DC392
:100110009840E198EB33FB0582E0FDC39CC3984017
:10012000D398EB33FB0582E0FCC39DC39840C59890
:10013000EB33FB0582E0FDC39CC39840B798EB33DB
:10014000FB0582E0FCC39DC39840A998EB33FB05F7
:1001500082E0FDC39CC398409B98EB33FB0582E093
:10016000FCC39DC398408D98EB33FB0582217890AA
:100170000000D2A8D2AA61E7E0FDC39CC39840EF7B
:1001800098EA33FA0582E0FCC39DC39840E198EAFF
:1001900033FA0582E0FDC39CC39840D398EA33FA52
:1001A0000582E0FCC39DC39840C598EA33FA0582F6
:1001B000E0FDC39CC39840B798EA33FA0582E0FC9F
:1001C000C39DC39840A998EA33FA0582E0FDC39C19
:1001D000C398409B98EA33FA0582E0FCC39DC3981C
:1001E000408D98EA33FA0582EBC46B6A54F0F9EA61
:1001F000C454F0C3996009900000D2A8D2AA61E764
:10020000EBF4C454F0F9EAF4C4540F49FAEBF4C423
:10021000540FFBC3EAF99460FAEB9400FB5020C33F
:10022000E97B007A0079006016C3135006F9C39584
:1002300052600AE9F5527553007900800205533087
:100240003A27C3EA94D0F8EB9407F9400BE8FAE9AF
:10025000FB203509D235415D303502C235203902E7
:10026000B235C3EA33FAEB33FBEB2B3B3BF9C3EB81
:1002700013FBEA13FAEA29FAEB3400FB30E3047AC1
:10028000FF7BFFE5255403601B202A18E55D33F949
:10029000EB7007C3E99A4002E9FAE53CC4332AFA55
:1002A000EB3400FBC3EA33C4540FF8EB33C454F00F
:1002B00048F87005EA60027801900000D2A8D2AA3E
:1002C000E5226002152281D4900000D2A8D2AA6152
:1002D000E7C0D0C0E0C2CF0541E5666009E56560D2
:1002E000057565006104756501E52360021523C38A
:1002F000E55460057555006104E5552401F5555038
:10030000037555FFD0E0D0D032C2AF53E67F75926F
:10031000FA7593FFC22053917FD2AF32C0E0E58AD5
:10032000303408856B8BF0A3D0E032D0E0C2AF53FD
:10033000E6EFC0D0C0E0C0F0D2D3D2AF5388EFA870
:100340008AA98CAA40308D010A758A00758C0075C7
:100350004000438810E566700AC3E833F8E933F9D2
:10036000EA33FA30331FE8C4540FFAE9C454F04AB0
:10037000FAC3132AFAC3E833F8E933F9E82AFAE9A9
:100380003406FB61D830320FC3E833E933FAE82A88
:10039000FAE93400FB61D8303115E875F056A4AAAB
:1003A000F0E975F056A42AFAC5F03400FB61D8C311
:1003B000EA13FAE913F9E813F8E875F056A4AAF07D
:1003C000E975F056A42AFAC5F03400C313FBEA130A
:1003D000FAC3EB13FBEA13FAC3EB94125009C3EA16
:1003E0009434EB940750160522E52270021522C3BF
:1003F000E52294325002A128755400A12BE5226019
:100400000215223036067C007D088117AC31AD32F2
:10041000303A04AC33AD34C3EA9CFAEB9DFB92084E
:10042000AE60AF61303A425007203509D235813590
:10043000303502C235303504AE62AF63203902B2C6
:1004400035C3EA33FAEB33FBA208500AEAF424017D
:10045000FAEBF43400FBC3EA9450FAEB9400FB503F
:100460001478007A007B008175A208500878007A21
:10047000007B0081D4E5255403601B202A18E55D2C
:1004800033F9EB7007C3E99A4002E9FAE53CC4335B
:100490002AFAEB3400FBEA8EF0A4F9AAF0EB8EF016
:1004A000A42AFAC5F03400FBC3EB13FDEA13F8C32A
:1004B000ED13FDE813F80FEF146004C3E833F8C33D
:1004C000E933EA33FAEB33FBDFEDEB30E30678FF99
:1004D0007AFF7B078854D230E86003755500C3E586
:1004E0005BFC955C4002AC5CC3EC95545008EC7529
:1004F000F008A4FAABF0EAF4F8EBF45407F9C3E817
:100500009450FAE99400FB50047A007B00885689E5
:10051000578A588B5975230AD0F0D0E0D0D053F7C2
:10052000DF43F74043E6103275230AD0F0D0E0D025
:10053000D043E61032C2AAD28EC2CA85CC6C85CD19
:100540006DD2CA32C2AFC0D0C0E0D2D3A8F9E55A4A
:1005500030E20AE5FA20E23520E132A165E5FA3021
:10056000E22B20E128C3E55713F8E55613F5FB8885
:10057000FCC3E55913F8E55813F5E988EA85575A9D
:1005800053F7BFD2A8303402D2AA53E6EF53F7DFB5
:10059000D0E0D0D0D2AF32790180147903801079C5
:1005A0000A800C791E80087964800479C8800078FC
:1005B00017E4D5E0FDD8FAD9F62278FF202828796B
:1005C000A1E76023E548601F74FF8548F084853FFC
:1005D000F030290375F005A4F8C5F0600278FFC378
:1005E000E8955D5002A85D885C22C3E54794A0E5CC
:1005F000489400E55C500314A1FB046002F55C2202
:1006000075E89022055EC3E55E9408405330EDF432
:10061000A8BDA9BE755E00E9FA79A0E76041EA705D
:1006200006E55F6018800CC3E8955F600EE55F50DB
:1006300005600A1480070460FA8002E55FF55FC375
:100640009569401B755BC0C394044013755B80C300
:100650009404400B755B40C394044003755B002217
:10066000E55B2410500274FFF55B22743279A68793
:10067000F0A4C5F0A2F733F55D227547007548F088
:1006800022C2AFC2CAA8CCA9CDAA4130CF010AD29A
:10069000CAD2AFC3EA13FAE913F9E813F8AB42ACD4
:1006A0004388428943C3E89BF8E99C20280A547F89
:1006B000F9302C02E19FC1F8AD448A44F9EA9D5417
:1006C0007FFA600678FF79FFC1DDAE45AF468B4506
:1006D0008C46A842A943C3E89EF8E99FF9C3E548C0
:1006E00013FBE54713FAE82AF547E93BF5485006BE
:1006F0007547FF7548FFE145AA47AB48AC47AD4891
:100700007E047F02C3EB9404400D1E1FC3EB9408CC
:1007100040052029021E1FC3ED13FDEC13FCDEF77C
:10072000C3EA9CFAEB9DFBEF6009C3E913F9E813F8
:10073000F8DFF7EA28FAEB39FB8A478B4850067B4B
:10074000FF8B478B48C3EB94025002D22C30280415
:100750007F03E1707892E6FFC3E53D948240110F7C
:10076000C3E53D94A040010FC3EF940640027F050E
:100770007E02E548C4540FF9E548C454F0F8E54753
:10078000C4540F28F8C3E89EFAE99400FB4009C35B
:10079000EA9401EB940050047A01E4FB0207EBAA0F
:1007A00047AB48EBC4FEEAC4540F4EFCC3EA9CFAC4
:1007B000EB9400FBC3E813C313F8EA28FAEB340008
:1007C000FB8A478B48C3EB94024002C22C7802EBB1
:1007D000C4FE7B00EAC4540F4EFAC3EA98FA4005FF
:1007E000C3940150027A017892E6FF302002E1EBD7
:1007F000854E92854F93D22043E680C3E49AF8E475
:100800009BF9C3E833F8E933F9302C03020880E898
:10081000FAE9FBD3E913FDE813FC884E894FC3EFD7
:1008200094036038EF20E00CE82CF8E93DF9ECFA8D
:10083000EDFB8013E828F8E939F9C3E82401F8E969
:100840003400F97AFF7BFFC3EF9403400F8A508B8B
:1008500051884A894B8C4C8D4D0208B5885089517E
:100860008A4A8B4B8C4C8D4D3028127550F0755147
:10087000FF754CF0754DFF754EF0754FFF0208B5D2
:10088000E8FAD3E813FC884EC3EF94036021EF200D
:10089000E007E82CF8ECFA01A0E8282401F87AFF38
:1008A000C3EF940340098A50884A8C4C0208B588EB
:1008B000508A4A8C4C30200201B5753A02D220434E
:1008C000E680E5255403602DA847A948C3E913F93C
:1008D000E813F8302804E92440F9C2AF53E67F75E5
:1008E0009100C3E498F594E499F595759104D220AC
:1008F00043E680D2AF22D221754900752000302B0B
:10090000037520402114D221754900752040302BF9
:100910000375200078017901202C20E5255403601F
:1009200002C2217914E548C313700104F8C394147A
:1009300040027814302804781B791BC3E833F8C3CD
:10094000E933F9202010E549600C302803D53A043A
:10095000D22221C711BD0549E59B5440B520022193
:10096000B130280908C3E899400118214320210A21
:1009700008C3E899400221142143C22153E67F7540
:100980009100302C117594007595F0759104D2206A
:1009900043E680020914E5487EFFC3334009C333B0
:1009A0004005C3334001FEC3E49E759400F59521D4
:1009B0008BC3E5399401500221143021022114D84F
:1009C0000221C52143C222C2AF53E67F7591008543
:1009D0005094855195759104854A92854B93D22008
:1009E00043E680D2AFE5255403600720290205398C
:1009F000801030220D202B0A20210715811581023D
:100A000013F52278003021027801E53D75F007A446
:100A1000F9E5F028F5F0E9A2F013A2F113A2F21320
:100A2000F53DC394785003753D78C3E53D953E4050
:100A300009C290C292C29475D57F302002413A8596
:100A40004C92854D93D22043E68022203810C2AFCD
:100A5000C293D29175D54FD2AF759F20611BC2AFA3
:100A6000C293D29575D57CD2AF759F20611B20387B
:100A700010C2AFC29475D573D291D2AF759F306159
:100A80001BC2AFC29075D573D295D2AF759F10615E
:100A90001B203810C2AFC291D29575D573D2AF75F5
:100AA0009F108077C2AFC295D29175D573D2AF75C2
:100AB0009F308067203810C2AFC29275D57CD29526
:100AC000D2AF759F208054C2AFC29275D54FD291DC
:100AD000D2AF759F208044203810C2AFC295D29308
:100AE00075D57CD2AF759F308031C2AFC291D293A1
:100AF00075D54FD2AF759F108021203810C2AFC27C
:100B00009075D54FD293D2AF759F10800EC2AFC2F1
:100B10009475D57CD293D2AF759F30227A147B78AE
:100B200080127A107B8C800C7A0D7BB480067A0B55
:100B30007BC88000E564D5E001227902E4C293D548
:100B4000E0FDD292D5E0FDC292D5E0FDD293D5E092
:100B5000FDE920E002D29030E002D294E564D5E0D5
:100B6000FDE920E002C29030E002C2947496D5E024
:100B7000FDD9C9EAF8D5E0FDD8FBDBB8C29322C2A3
:100B800090C292C294C291C293C29575D57F2278C9
:100B90008076FF0876FF0876FF0876FF0876FF0864
:100BA00076FF0876090876FF087601788C760108CA
:100BB00076FF0876FF0876FF0876FF0876FF08764E
:100BC000030876FF0876FF0876FF0876250876D0BA
:100BD0000876280876500876040876FF087602081A
:100BE00076FF08767A0876FF087607087601087699
:100BF000FF0876FF08760008760022FA75F00CA44C
:100C0000ABF0EAC333F8740133F9E8C333F8E933DE
:100C1000F9E8C32BF8E93400F9E8C333F8E933F90C
:100C2000227888E6C39403D23A5002C23AC238E628
:100C300030E102D238A23892397886E614900080EA
:100C40009378A6F67886E6F53FC394025003753F85
:100C500002789CE6753EFFB40203753EA0B4030320
:100C6000753E8278A0E6F8600674282409D8FCF561
:100C7000697896E671FB88318932789EE671FB8847
:100C80003389347897E671FB88358936717F223055
:100C900036117A007B007CFF7D007E0091F58B6130
:100CA0008A6022303A227896E6FA7B00789EE6FC4B
:100CB0007D00C3EA33FAEB33FBC3EC33FCED33FDC9
:100CC0007E0A91F58B638A627896303A02789EE6C6
:100CD000FA7B007897E6FC7D007E00303A10C3EA8C
:100CE00033FAEB33FBC3EC33FCED33FD7E0A91F5B5
:100CF0008B618A6022C3EC9EFCED9400FDC3EC9AEC
:100D0000FCED9BFDC3EC9423ED940050047C237D0B
:100D100000C3EC94FFED940140047CFF7D017BFF58
:100D20000B7A000AEA7009C3EC33FCED33FDA12015
:100D3000EC8AF0A4AEF0ED8AF0A42E947C40E4EAB4
:100D4000F460DD22D236918F1205A31205A37A003A
:100D50007B007C1012059BE5542AFA74003BFBDCF7
:100D6000F37C04C3EB13FBEA13FADCF7FFEB60023E
:100D70007FFFC236918F2278A5E6F95403D28670A0
:100D800002C286E9540CD2877002C287E95430D27D
:100D9000967002C296E954C07000227567007568AB
:100DA000007597DE7597AD7581C043FF8075EF06BE
:100DB00075A900717F75803F75F1F075A4C07580CD
:100DC0003F75D4FF75900075F27F75A57F75900013
:100DD00075D57F75A60175E34075E202C290C29297
:100DE000C2941205A7D291D293D295120597C291BF
:100DF000C293C295717FE4F8F6D8FD718F12143951
:100E000078988664753001C2AF1205AB711C12056B
:100E1000A371221205A371281205A3B177C2AF7581
:100E2000670075680078FA79FA308507D9FBD8F73A
:100E3000021C009121918F78988664717F75A913A7
:100E400075A71075C10075A70075660075E4057576
:100E50008811758E0475890975C80475910475D853
:100E60004075D90875F782759E0375960275DA424A
:100E700075DB4275A82375E69075B801759B807582
:100E80009D0075D10C75BCB975BB1075E88075B245
:100E900001120597D2AF753C00C2301205ABC231CA
:100EA000C232C233C234755200755300752200122B
:100EB00005A7C3E522940A5002E183D231752200CE
:100EC0001205A7C3E522940A5002E183C231D2324F
:100ED0007522001205A7C3E522940A5002E183752A
:100EE000E4D5758851758E017589AA758C00758D4C
:100EF00000C2A9D2ABD2AA756B80756A14756E5008
:100F0000C232D23475220A1205A7756A10C3E522CF
:100F1000940A7552007553004069758E0C756B000C
:100F2000756A28756E2875220A1205A7756A20C38E
:100F3000E522940A7552007553004047758E0C7572
:100F40006B80756A14756E1475220A1205A7756A8E
:100F500010C3E522940A755200755300402575E4CC
:100F600005758811758E04758909D2A9C2ABC2AA0C
:100F7000C234D2337522001205A7C3E522940A4079
:100F800002C11D12059B203003020E1DC2AF711C51
:100F9000711C711CD2AF1205AB203403303A03022E
:100FA000104512059B788CE6C3940150030210454E
:100FB000E530C3940150030210457567A57568F1CB
:100FC0007F02D236918F1205A7C2AFC236918FC36E
:100FD000E554947FD2AF406D120597C2AF712ED207
:100FE000AFDFDFB144C3EF7897F61205AB121526D9
:100FF0007F0AD236918F1205A7C2AFC236918FC336
:10100000E554947FD2AF50E8120597C2AF120B1C83
:1010100012059F120B1CD2AFDFD8120D44EF240330
:101020007896F6F87997E7C394234003985006E83A
:1010300024237897F61205AB9180B1551205A712BB
:101040000C8F020E1D7567007568001205A7C3E5B9
:101050005494014003020F99C2AF120B2E120B2EB3
:10106000120B2ED2AF1205AB753000E4F537F53810
:101070000537E537F4703F0538789AE6781914603B
:1010800012783214600D787D14600878FA146003C9
:10109000753800C3E53898401D120B7F120597156F
:1010A0003875370078998664C2AF120B2ED2AF78AC
:1010B0009886641205A712059FE5237003020E1D92
:1010C000C3E5549401500AC3E5529401501602102E
:1010D000701205A7E5237003020E1D7552007553AB
:1010E00000021286C3E55294017017C2AF120B7F43
:1010F00078998664120B1C78988664D2AF1205A783
:101100004178C3E55294027017C2AF120B7F7899F1
:101110008664120B2278988664D2AF1205A74178B4
:10112000C3E55294037017C2AF120B7F789986649F
:10113000120B2878988664D2AF1205A74178C3E5D0
:101140005294047017C2AF120B7F78998664120B09
:101150002E78988664D2AF1205A74178C3E55294E1
:10116000057017C2AF120B7F78998664120B2E7828
:10117000988664D2AF1205A74178C3E552940770F0
:1011800019C3E5539406500201C07401303A027449
:10119000037888F6C238C2394178C3E552940870A2
:1011A00019C3E5539406500201C07402303A027428
:1011B000047888F6D238D2394178C3E55294097060
:1011C00017C3E5539406500201C0303A0BC3788828
:1011D000E69402F6C23A4178C3E552940A7016C307
:1011E000E5539406500201C0203A0A7888E62402AA
:1011F000F6D23A4178C3E55294147025C3E553946E
:1012000006500201C0C2AF901A0B740093D2AF789F
:1012100088F613C238C2394002D2384002D239802F
:1012200057C3E55294157038C3E5539406404FC236
:10123000AF901A0B740093D2AFF8B801027402B8E1
:1012400002027401B803027404B8040274037888BB
:10125000F613C238C2394002D2384002D23980185F
:10126000C3E552940C70117567A57568F1C3E55319
:101270009406400A9180D2AF75520075530075678D
:101280000075680001C0C2AF120B7FE4D2AFE4F575
:101290005EF524F525F53D755E08120597120600EA
:1012A00030EDFDA8BDA9BEE97001F8885F12060403
:1012B000755E08C2AF12066B855D5B855D5CD2AF63
:1012C00075A71075C13075A70075A9037566013043
:1012D0003A07C238303502D238D228753900120A9E
:1012E000D7120AFA12067A12068112067A120681BB
:1012F00012067A120906120A03120A4B120681120A
:1013000008F6202C031205BA302C031205EA120A43
:1013100003120A6E120681120906120A03120A91BA
:101320001206811208F6120A03120AB4120681127A
:101330000906120A03120AD71206811206001208C1
:10134000F6120A03120AFA1206041206813028273E
:10135000855D5B79187A0CC3E53999400EC228D2B5
:10136000298A3B855D5B855D5C800CC3E5549401F7
:1013700040030212F361FD30291F202B1CE53B14B2
:101380007006C229D22A41F3F53B203A07C3E5543F
:10139000940140030212F38064753C00203A0F78F8
:1013A000FA79A4E760027803C3E55598504FE52326
:1013B000604B303A17203805203507800F30350252
:1013C000800A202B07D22B855D5B612378F0302BC0
:1013D00005855D5B7820C3E5489850030212F33021
:1013E0002B1BC22BC238303502D238D229753B12A2
:1013F000855D5B41F3053CE55460028100753C006E
:10140000C2AF120B7F75240075250075A91375A74F
:101410001075C10075A700756600D2AF1205A7123E
:101420000B7F78A4E66006D291D293D295C3E53CB7
:1014300094044003020E1D016B901A0D782091B99F
:10144000E520B4550AA391B9E520B4AA028013752A
:1014500067A57568F1120B8F91807567007568003C
:10146000801D901A0378807B0A91B9A308DBFA905B
:101470001A0F788C7B1A91B9A308DBFA901A2922EB
:10148000C2AF91FC91D9901A00741091BEA3740759
:1014900091BEA3742191BE901A0378807B0A91BDFE
:1014A000A308DBFA901A0F788C7B1A91BDA308DB96
:1014B000FAB10F91ED901A2922E493F622E6438FB8
:1014C00001538FFDFFC3E583941C400122EF856724
:1014D000B78568B7F0538FFE22438F02438F018593
:1014E00067B78568B7901A0DF0538FFC22901A0DDC
:1014F000745591BE901A0E74AA91BE227A3079D09A
:101500007820901A4091B9E520F709A3DAF7227AFA
:101510003079D0901A40E791BE09A3DAF9227C0510
:101520001205ABDCFB22C2AF120B1C120B22120BFA
:1015300028120B2E12059F120B1C120B22120B28C5
:10154000120B2E12059F120B1C120B22120B2812CB
:101550000B2ED2AF22C2AF120B2E120B28120B226F
:10156000120B1C12059F120B2E120B28120B2212AB
:101570000B1C12059F120B2E120B28120B22120BA2
:041580001CD2AF22A8
:1019FD00020D9B100721FFFFFFFFFFFF09FF01FFF6
:101A0D0055AA01FFFFFFFFFF03FFFFFF25D0285061
:0D1A1D0004FF02FF7AFF0701FFFF0000FF3A
:101A400023455F485F3430232020202020202020A1
:101A500023424C48454C492445464D3842323123B7
:101A60002020202020202020202020202020202076
:101C0000C2AFC2D37597DE7597AD7581C075A90057
:101C100043FF80752438752503B1DB7529A5752A26
:101C2000F143F12053A4DFD28575D4FF75E3407DE5
:101C3000FA780379E67C10752200752300901DE880
:101C40007B0675249875250130850281482085081A
:101C5000D8FBD9F9DCF781BA308508D8FBD9F9DC93
:101C6000F781BAB19BE493A3C39A6004DDC381BA40
:101C7000DBDBB18D600281317B08E493FAA3B16EA6
:101C8000DBF87A30B16E752200752300B18DEAFC65
:101C9000EBFDC3ED94FE400EB18D8A278B28ED300D
:101CA000E0048A828B83B18D7AC270D8C3ED94FE32
:101CB000601950CEBD0029EC600F7520007521FF22
:101CC000752900752A000200008100A827A92808AC
:101CD00009D804D90281DDB191EAF281D10D81A642
:101CE000C3ED94035051EDA2E092007AC5C3E582A2
:101CF0009400E583941C508C200010438F02438F86
:101D0000018529B7852AB7F0300027A827A9280818
:101D100009438F01538FFDD804D902A132C3E58353
:101D2000941C4003A3A117E28529B7852AB7F0A325
:101D3000A117538FFC81827AC1BD030CE493A3FAEF
:101D4000B152DCF8B14A81828184AA22AB23B16E00
:101D5000EBFAEA6222752608C3E52313F523E52290
:101D600013F52250066323A0632201D526EAB1DBD6
:101D7000B1DB75260AEAF4200102D285300102C2E5
:101D800085B1DBC3134002C201D526EB22B191EA33
:101D9000FB208502A191308502A196752608AE240C
:101DA000AF25C3EF13FFEE13FEB1DFB1DBC3EA13C0
:101DB0003085024480FA30E703632201C3E5231330
:101DC000F523E52213F52250066323A0632201D5F3
:101DD00026D9E52265236523F52222AE24AF250E00
:101DE0000FDEFEDFFCD20122424C48656C693437BD
:061DF0003164E8B20601B7
:00000001FF
